
 Start         Length     Name                   Class
 0001:00401000 00005994H .text                   CODE
 0002:00407000 0000029CH .itext                  ICODE
 0003:00408000 00000040H .data                   DATA
 0004:00409000 00000038H .bss                    BSS
 0005:00000000 00000000H .tls                    TLS


Detailed map of segments

 0001:00000000 00000146 C=CODE     S=.text    G=(none)   M=System   ACBP=A9
 0001:00000148 0000005C C=CODE     S=.text    G=(none)   M=Windows  ACBP=A9
 0001:000001A4 0000003E C=CODE     S=.text    G=(none)   M=SysUtils ACBP=A9
 0001:000001E4 00000006 C=CODE     S=.text    G=(none)   M=ActnList ACBP=A9
 0001:000001EC 00000096 C=CODE     S=.text    G=(none)   M=Classes  ACBP=A9
 0001:00000284 00000016 C=CODE     S=.text    G=(none)   M=TypInfo  ACBP=A9
 0001:0000029C 00000006 C=CODE     S=.text    G=(none)   M=Variants ACBP=A9
 0001:000002A4 00000006 C=CODE     S=.text    G=(none)   M=VarUtils ACBP=A9
 0001:000002AC 00000006 C=CODE     S=.text    G=(none)   M=Graphics ACBP=A9
 0001:000002B4 00000006 C=CODE     S=.text    G=(none)   M=Registry ACBP=A9
 0001:000002BC 00000006 C=CODE     S=.text    G=(none)   M=IniFiles ACBP=A9
 0001:000002C4 00000006 C=CODE     S=.text    G=(none)   M=Themes   ACBP=A9
 0001:000002CC 00000186 C=CODE     S=.text    G=(none)   M=Controls ACBP=A9
 0001:00000454 00000006 C=CODE     S=.text    G=(none)   M=Menus    ACBP=A9
 0001:0000045C 00000006 C=CODE     S=.text    G=(none)   M=UxTheme  ACBP=A9
 0001:00000464 00000006 C=CODE     S=.text    G=(none)   M=MultiMon ACBP=A9
 0001:0000046C 00000006 C=CODE     S=.text    G=(none)   M=DwmApi   ACBP=A9
 0001:00000474 0000012E C=CODE     S=.text    G=(none)   M=Forms    ACBP=A9
 0001:000005A4 00000006 C=CODE     S=.text    G=(none)   M=HelpIntfs ACBP=A9
 0001:000005AC 0000000E C=CODE     S=.text    G=(none)   M=Dialogs  ACBP=A9
 0001:000005BC 00000006 C=CODE     S=.text    G=(none)   M=Printers ACBP=A9
 0001:000005C4 0000000E C=CODE     S=.text    G=(none)   M=ExtCtrls ACBP=A9
 0001:000005D4 00000006 C=CODE     S=.text    G=(none)   M=GraphUtil ACBP=A9
 0001:000005DC 00000006 C=CODE     S=.text    G=(none)   M=Clipbrd  ACBP=A9
 0001:000005E4 00000006 C=CODE     S=.text    G=(none)   M=FlatSB   ACBP=A9
 0001:000005EC 000000FE C=CODE     S=.text    G=(none)   M=DesignEditors ACBP=A9
 0001:000006EC 0000000E C=CODE     S=.text    G=(none)   M=DesignIntf ACBP=A9
 0001:000006FC 00000006 C=CODE     S=.text    G=(none)   M=ToolsAPI ACBP=A9
 0001:00000704 00000006 C=CODE     S=.text    G=(none)   M=XMLIntf  ACBP=A9
 0001:0000070C 00000006 C=CODE     S=.text    G=(none)   M=xmldom   ACBP=A9
 0001:00000714 00000006 C=CODE     S=.text    G=(none)   M=msxmldom ACBP=A9
 0001:0000071C 00000006 C=CODE     S=.text    G=(none)   M=ComObj   ACBP=A9
 0001:00000724 00000006 C=CODE     S=.text    G=(none)   M=ComCtrls ACBP=A9
 0001:0000072C 00000006 C=CODE     S=.text    G=(none)   M=ExtActns ACBP=A9
 0001:00000734 00000006 C=CODE     S=.text    G=(none)   M=ExtDlgs  ACBP=A9
 0001:0000073C 00000006 C=CODE     S=.text    G=(none)   M=Buttons  ACBP=A9
 0001:00000744 00000006 C=CODE     S=.text    G=(none)   M=Mapi     ACBP=A9
 0001:0000074C 00000006 C=CODE     S=.text    G=(none)   M=DockForm ACBP=A9
 0001:00000754 00000006 C=CODE     S=.text    G=(none)   M=IDEMessages ACBP=A9
 0001:0000075C 00000006 C=CODE     S=.text    G=(none)   M=DeskForm ACBP=A9
 0001:00000764 00000006 C=CODE     S=.text    G=(none)   M=BaseDock ACBP=A9
 0001:0000076C 00000006 C=CODE     S=.text    G=(none)   M=PercentageDockTree ACBP=A9
 0001:00000774 00000006 C=CODE     S=.text    G=(none)   M=CaptionedDockTree ACBP=A9
 0001:0000077C 00000006 C=CODE     S=.text    G=(none)   M=DockTabSet ACBP=A9
 0001:00000784 00000006 C=CODE     S=.text    G=(none)   M=Tabs     ACBP=A9
 0001:0000078C 00000006 C=CODE     S=.text    G=(none)   M=DeskUtil ACBP=A9
 0001:00000794 00000006 C=CODE     S=.text    G=(none)   M=ActnMan  ACBP=A9
 0001:0000079C 00000006 C=CODE     S=.text    G=(none)   M=ActnMenus ACBP=A9
 0001:000007A4 00000006 C=CODE     S=.text    G=(none)   M=XPStyleActnCtrls ACBP=A9
 0001:000007AC 00000006 C=CODE     S=.text    G=(none)   M=Proxies  ACBP=A9
 0001:000007B4 0000002E C=CODE     S=.text    G=(none)   M=ovcsf    ACBP=A9
 0001:000007E4 0000000E C=CODE     S=.text    G=(none)   M=ovcdata  ACBP=A9
 0001:000007F4 00000006 C=CODE     S=.text    G=(none)   M=o32sr    ACBP=A9
 0001:000007FC 00000006 C=CODE     S=.text    G=(none)   M=ovcdate  ACBP=A9
 0001:00000804 00000006 C=CODE     S=.text    G=(none)   M=ovcstr   ACBP=A9
 0001:0000080C 00000026 C=CODE     S=.text    G=(none)   M=ovcbase  ACBP=A9
 0001:00000834 00000016 C=CODE     S=.text    G=(none)   M=ovcintl  ACBP=A9
 0001:0000084C 000000EE C=CODE     S=.text    G=(none)   M=ovcef    ACBP=A9
 0001:0000093C 00000006 C=CODE     S=.text    G=(none)   M=ovccalc  ACBP=A9
 0001:00000944 00000006 C=CODE     S=.text    G=(none)   M=ovcuser  ACBP=A9
 0001:0000094C 00000006 C=CODE     S=.text    G=(none)   M=ovcrptvw ACBP=A9
 0001:00000954 00000006 C=CODE     S=.text    G=(none)   M=ovcrvexpdef ACBP=A9
 0001:0000095C 00000006 C=CODE     S=.text    G=(none)   M=ovcfxfnt ACBP=A9
 0001:00000964 0000000E C=CODE     S=.text    G=(none)   M=ovctcnum ACBP=A9
 0001:00000974 0000000E C=CODE     S=.text    G=(none)   M=ovctcbef ACBP=A9
 0001:00000984 00000026 C=CODE     S=.text    G=(none)   M=ovctbcls ACBP=A9
 0001:000009AC 00000006 C=CODE     S=.text    G=(none)   M=o32rxvld ACBP=A9
 0001:000009B4 00000006 C=CODE     S=.text    G=(none)   M=o32vlreg ACBP=A9
 0001:000009BC 00000006 C=CODE     S=.text    G=(none)   M=o32pvldr ACBP=A9
 0001:000009C4 00000006 C=CODE     S=.text    G=(none)   M=o32ovldr ACBP=A9
 0001:000009CC 00000016 C=CODE     S=.text    G=(none)   M=ovctcpic ACBP=A9
 0001:000009E4 00000016 C=CODE     S=.text    G=(none)   M=ovctcsim ACBP=A9
 0001:000009FC 00000006 C=CODE     S=.text    G=(none)   M=ovctgres ACBP=A9
 0001:00000A04 000001C3 C=CODE     S=.text    G=(none)   M=SysInit  ACBP=A9
 0001:00000BC8 0000001E C=CODE     S=.text    G=(none)   M=ovcdbsf  ACBP=A9
 0001:00000BE8 00000006 C=CODE     S=.text    G=(none)   M=DBCtrls  ACBP=A9
 0001:00000BF0 0000000E C=CODE     S=.text    G=(none)   M=DB       ACBP=A9
 0001:00000C00 00000006 C=CODE     S=.text    G=(none)   M=WideStrings ACBP=A9
 0001:00000C08 00000006 C=CODE     S=.text    G=(none)   M=FMTBcd   ACBP=A9
 0001:00000C10 00000006 C=CODE     S=.text    G=(none)   M=SqlTimSt ACBP=A9
 0001:00000C18 00000006 C=CODE     S=.text    G=(none)   M=DBPWDlg  ACBP=A9
 0001:00000C20 00000006 C=CODE     S=.text    G=(none)   M=DBLogDlg ACBP=A9
 0001:00000C28 00000066 C=CODE     S=.text    G=(none)   M=ovcdbae  ACBP=A9
 0001:00000C90 00000BAE C=CODE     S=.text    G=(none)   M=ovcdbae0 ACBP=A9
 0001:00001840 000005DA C=CODE     S=.text    G=(none)   M=ovcdbae1 ACBP=A9
 0001:00001E1C 0000087A C=CODE     S=.text    G=(none)   M=ovcdbae2 ACBP=A9
 0001:00002698 000007BE C=CODE     S=.text    G=(none)   M=ovcdbae3 ACBP=A9
 0001:00002E58 00000006 C=CODE     S=.text    G=(none)   M=BDE      ACBP=A9
 0001:00002E60 0000005E C=CODE     S=.text    G=(none)   M=DBTables ACBP=A9
 0001:00002EC0 00000426 C=CODE     S=.text    G=(none)   M=ovcdbhbd ACBP=A9
 0001:000032E8 0000003E C=CODE     S=.text    G=(none)   M=ovcdbtbl ACBP=A9
 0001:00003328 0000033A C=CODE     S=.text    G=(none)   M=ovcdbtb1 ACBP=A9
 0001:00003664 0000149A C=CODE     S=.text    G=(none)   M=ovcdbtb0 ACBP=A9
 0001:00004B00 0000005E C=CODE     S=.text    G=(none)   M=ovcregbd ACBP=A9
 0001:00004B60 000005F2 C=CODE     S=.text    G=(none)   M=ovcregdb ACBP=A9
 0001:00005154 0000083F C=CODE     S=.text    G=(none)   M=.O406BD2005 ACBP=A9
 0002:00000000 00000006 C=ICODE    S=.itext   G=(none)   M=System   ACBP=A9
 0002:00000008 00000011 C=ICODE    S=.itext   G=(none)   M=Windows  ACBP=A9
 0002:0000001C 00000006 C=ICODE    S=.itext   G=(none)   M=SysUtils ACBP=A9
 0002:00000024 00000006 C=ICODE    S=.itext   G=(none)   M=ActnList ACBP=A9
 0002:0000002C 00000006 C=ICODE    S=.itext   G=(none)   M=Classes  ACBP=A9
 0002:00000034 00000006 C=ICODE    S=.itext   G=(none)   M=TypInfo  ACBP=A9
 0002:0000003C 00000006 C=ICODE    S=.itext   G=(none)   M=Variants ACBP=A9
 0002:00000044 00000006 C=ICODE    S=.itext   G=(none)   M=VarUtils ACBP=A9
 0002:0000004C 00000006 C=ICODE    S=.itext   G=(none)   M=Graphics ACBP=A9
 0002:00000054 00000006 C=ICODE    S=.itext   G=(none)   M=Registry ACBP=A9
 0002:0000005C 00000006 C=ICODE    S=.itext   G=(none)   M=IniFiles ACBP=A9
 0002:00000064 00000006 C=ICODE    S=.itext   G=(none)   M=Themes   ACBP=A9
 0002:0000006C 00000006 C=ICODE    S=.itext   G=(none)   M=Controls ACBP=A9
 0002:00000074 00000006 C=ICODE    S=.itext   G=(none)   M=Menus    ACBP=A9
 0002:0000007C 00000006 C=ICODE    S=.itext   G=(none)   M=UxTheme  ACBP=A9
 0002:00000084 00000006 C=ICODE    S=.itext   G=(none)   M=MultiMon ACBP=A9
 0002:0000008C 00000006 C=ICODE    S=.itext   G=(none)   M=DwmApi   ACBP=A9
 0002:00000094 00000006 C=ICODE    S=.itext   G=(none)   M=Forms    ACBP=A9
 0002:0000009C 00000006 C=ICODE    S=.itext   G=(none)   M=HelpIntfs ACBP=A9
 0002:000000A4 00000006 C=ICODE    S=.itext   G=(none)   M=Dialogs  ACBP=A9
 0002:000000AC 00000006 C=ICODE    S=.itext   G=(none)   M=Printers ACBP=A9
 0002:000000B4 00000006 C=ICODE    S=.itext   G=(none)   M=ExtCtrls ACBP=A9
 0002:000000BC 00000006 C=ICODE    S=.itext   G=(none)   M=GraphUtil ACBP=A9
 0002:000000C4 00000006 C=ICODE    S=.itext   G=(none)   M=Clipbrd  ACBP=A9
 0002:000000CC 00000006 C=ICODE    S=.itext   G=(none)   M=FlatSB   ACBP=A9
 0002:000000D4 00000006 C=ICODE    S=.itext   G=(none)   M=DesignEditors ACBP=A9
 0002:000000DC 00000006 C=ICODE    S=.itext   G=(none)   M=ToolsAPI ACBP=A9
 0002:000000E4 00000006 C=ICODE    S=.itext   G=(none)   M=XMLIntf  ACBP=A9
 0002:000000EC 00000006 C=ICODE    S=.itext   G=(none)   M=xmldom   ACBP=A9
 0002:000000F4 00000006 C=ICODE    S=.itext   G=(none)   M=msxmldom ACBP=A9
 0002:000000FC 00000006 C=ICODE    S=.itext   G=(none)   M=ComObj   ACBP=A9
 0002:00000104 00000006 C=ICODE    S=.itext   G=(none)   M=ComCtrls ACBP=A9
 0002:0000010C 00000006 C=ICODE    S=.itext   G=(none)   M=ExtActns ACBP=A9
 0002:00000114 00000006 C=ICODE    S=.itext   G=(none)   M=ExtDlgs  ACBP=A9
 0002:0000011C 00000006 C=ICODE    S=.itext   G=(none)   M=Buttons  ACBP=A9
 0002:00000124 00000006 C=ICODE    S=.itext   G=(none)   M=Mapi     ACBP=A9
 0002:0000012C 00000006 C=ICODE    S=.itext   G=(none)   M=DockForm ACBP=A9
 0002:00000134 00000006 C=ICODE    S=.itext   G=(none)   M=IDEMessages ACBP=A9
 0002:0000013C 00000006 C=ICODE    S=.itext   G=(none)   M=DeskForm ACBP=A9
 0002:00000144 00000006 C=ICODE    S=.itext   G=(none)   M=BaseDock ACBP=A9
 0002:0000014C 00000006 C=ICODE    S=.itext   G=(none)   M=PercentageDockTree ACBP=A9
 0002:00000154 00000006 C=ICODE    S=.itext   G=(none)   M=CaptionedDockTree ACBP=A9
 0002:0000015C 00000006 C=ICODE    S=.itext   G=(none)   M=DockTabSet ACBP=A9
 0002:00000164 00000006 C=ICODE    S=.itext   G=(none)   M=Tabs     ACBP=A9
 0002:0000016C 00000006 C=ICODE    S=.itext   G=(none)   M=DeskUtil ACBP=A9
 0002:00000174 00000006 C=ICODE    S=.itext   G=(none)   M=ActnMan  ACBP=A9
 0002:0000017C 00000006 C=ICODE    S=.itext   G=(none)   M=ActnMenus ACBP=A9
 0002:00000184 00000006 C=ICODE    S=.itext   G=(none)   M=XPStyleActnCtrls ACBP=A9
 0002:0000018C 00000006 C=ICODE    S=.itext   G=(none)   M=Proxies  ACBP=A9
 0002:00000194 00000006 C=ICODE    S=.itext   G=(none)   M=ovcdata  ACBP=A9
 0002:0000019C 00000006 C=ICODE    S=.itext   G=(none)   M=o32sr    ACBP=A9
 0002:000001A4 00000006 C=ICODE    S=.itext   G=(none)   M=ovcdate  ACBP=A9
 0002:000001AC 00000006 C=ICODE    S=.itext   G=(none)   M=ovcbase  ACBP=A9
 0002:000001B4 00000006 C=ICODE    S=.itext   G=(none)   M=ovcintl  ACBP=A9
 0002:000001BC 00000006 C=ICODE    S=.itext   G=(none)   M=ovccalc  ACBP=A9
 0002:000001C4 00000006 C=ICODE    S=.itext   G=(none)   M=ovcuser  ACBP=A9
 0002:000001CC 00000006 C=ICODE    S=.itext   G=(none)   M=ovcrptvw ACBP=A9
 0002:000001D4 00000006 C=ICODE    S=.itext   G=(none)   M=ovcrvexpdef ACBP=A9
 0002:000001DC 00000006 C=ICODE    S=.itext   G=(none)   M=ovcfxfnt ACBP=A9
 0002:000001E4 00000006 C=ICODE    S=.itext   G=(none)   M=o32rxvld ACBP=A9
 0002:000001EC 00000006 C=ICODE    S=.itext   G=(none)   M=o32vlreg ACBP=A9
 0002:000001F4 00000006 C=ICODE    S=.itext   G=(none)   M=o32pvldr ACBP=A9
 0002:000001FC 00000006 C=ICODE    S=.itext   G=(none)   M=o32ovldr ACBP=A9
 0002:00000204 00000006 C=ICODE    S=.itext   G=(none)   M=ovctgres ACBP=A9
 0002:0000020C 00000006 C=ICODE    S=.itext   G=(none)   M=DBCtrls  ACBP=A9
 0002:00000214 00000006 C=ICODE    S=.itext   G=(none)   M=DB       ACBP=A9
 0002:0000021C 00000006 C=ICODE    S=.itext   G=(none)   M=WideStrings ACBP=A9
 0002:00000224 00000006 C=ICODE    S=.itext   G=(none)   M=FMTBcd   ACBP=A9
 0002:0000022C 00000006 C=ICODE    S=.itext   G=(none)   M=SqlTimSt ACBP=A9
 0002:00000234 00000006 C=ICODE    S=.itext   G=(none)   M=DBPWDlg  ACBP=A9
 0002:0000023C 00000006 C=ICODE    S=.itext   G=(none)   M=DBLogDlg ACBP=A9
 0002:00000244 00000008 C=ICODE    S=.itext   G=(none)   M=ovcdbae0 ACBP=A9
 0002:0000024C 00000008 C=ICODE    S=.itext   G=(none)   M=ovcdbae1 ACBP=A9
 0002:00000254 00000008 C=ICODE    S=.itext   G=(none)   M=ovcdbae2 ACBP=A9
 0002:0000025C 00000008 C=ICODE    S=.itext   G=(none)   M=ovcdbae3 ACBP=A9
 0002:00000264 00000006 C=ICODE    S=.itext   G=(none)   M=DBTables ACBP=A9
 0002:0000026C 00000008 C=ICODE    S=.itext   G=(none)   M=ovcdbhbd ACBP=A9
 0002:00000274 00000008 C=ICODE    S=.itext   G=(none)   M=ovcdbtb1 ACBP=A9
 0002:0000027C 00000008 C=ICODE    S=.itext   G=(none)   M=ovcdbtb0 ACBP=A9
 0002:00000284 00000008 C=ICODE    S=.itext   G=(none)   M=ovcregbd ACBP=A9
 0002:0000028C 00000008 C=ICODE    S=.itext   G=(none)   M=ovcregdb ACBP=A9
 0002:00000294 00000005 C=ICODE    S=.itext   G=(none)   M=.O406BD2005 ACBP=A9
 0003:00000000 0000002C C=DATA     S=.data    G=DGROUP   M=SysInit  ACBP=A9
 0004:00000000 00000008 C=BSS      S=.bss     G=DGROUP   M=Windows  ACBP=A9
 0004:00000008 0000000C C=BSS      S=.bss     G=DGROUP   M=SysInit  ACBP=A9
 0004:00000014 00000004 C=BSS      S=.bss     G=DGROUP   M=ovcdbae0 ACBP=A9
 0004:00000018 00000004 C=BSS      S=.bss     G=DGROUP   M=ovcdbae1 ACBP=A9
 0004:0000001C 00000004 C=BSS      S=.bss     G=DGROUP   M=ovcdbae2 ACBP=A9
 0004:00000020 00000004 C=BSS      S=.bss     G=DGROUP   M=ovcdbae3 ACBP=A9
 0004:00000024 00000004 C=BSS      S=.bss     G=DGROUP   M=ovcdbhbd ACBP=A9
 0004:00000028 00000004 C=BSS      S=.bss     G=DGROUP   M=ovcdbtb1 ACBP=A9
 0004:0000002C 00000004 C=BSS      S=.bss     G=DGROUP   M=ovcdbtb0 ACBP=A9
 0004:00000030 00000004 C=BSS      S=.bss     G=DGROUP   M=ovcregbd ACBP=A9
 0004:00000034 00000004 C=BSS      S=.bss     G=DGROUP   M=ovcregdb ACBP=A9


  Address             Publics by Name

 0002:00000294       .O406BD2005..O406BD2005
 0001:00005974       .O406BD2005.@GetPackageInfoTable
 0001:0000597C       .O406BD2005.@PackageLoad
 0001:00005988       .O406BD2005.@PackageUnload
 0004:00000014       ovcdbae0..5
 0001:000011BC       ovcdbae0..TDbAeRangeProperty
 0001:00000EB8       ovcdbae0..TLocalAE
 0001:00001020       ovcdbae0..TLocalEF
 0001:00000C90       ovcdbae0..TOvcfrmDbAeRange
 0001:00001330       ovcdbae0.ChangeFromRange
 0001:00001398       ovcdbae0.ChangeToRange
 0001:00001810       ovcdbae0.Finalization
 0001:000013FC       ovcdbae0.GetDecimalPlaces
 0002:00000244       ovcdbae0.ovcdbae0
 0001:0000146C       ovcdbae0.TDbAeRangeProperty.Edit
 0001:00001294       ovcdbae0.TDbAeRangeProperty.GetAttributes
 0001:000012D8       ovcdbae0.TDbAeRangeProperty.GetValue
 0004:00000018       ovcdbae1..3
 0001:00001A64       ovcdbae1..TDbAeSimpleMaskProperty
 0001:00001840       ovcdbae1..TOvcfrmDbAeSimpleMask
 0001:00001DEC       ovcdbae1.Finalization
 0002:0000024C       ovcdbae1.ovcdbae1
 0001:00001C28       ovcdbae1.TDbAeSimpleMaskProperty.AllEqual
 0001:00001C2C       ovcdbae1.TDbAeSimpleMaskProperty.Edit
 0001:00001C1C       ovcdbae1.TDbAeSimpleMaskProperty.GetAttributes
 0001:00001DE4       ovcdbae1.TDbAeSimpleMaskProperty.GetEditLimit
 0001:00001BA8       ovcdbae1.TOvcfrmDbAeSimpleMask.cbxMaskCharacterChange
 0001:00001B44       ovcdbae1.TOvcfrmDbAeSimpleMask.FormCreate
 0004:0000001C       ovcdbae2..3
 0001:00002098       ovcdbae2..TDbAePictureMaskProperty
 0001:00001E1C       ovcdbae2..TOvcfrmDbAePictureMask
 0001:00002668       ovcdbae2.Finalization
 0002:00000254       ovcdbae2.ovcdbae2
 0001:00002188       ovcdbae2.TDbAePictureMaskProperty.AllEqual
 0001:0000218C       ovcdbae2.TDbAePictureMaskProperty.Edit
 0001:0000217C       ovcdbae2.TDbAePictureMaskProperty.GetAttributes
 0001:00002390       ovcdbae2.TOvcfrmDbAePictureMask.FormCreate
 0001:0000265C       ovcdbae2.TOvcfrmDbAePictureMask.FormDestroy
 0001:000025A4       ovcdbae2.TOvcfrmDbAePictureMask.lbMaskClick
 0004:00000020       ovcdbae3..3
 0001:00002914       ovcdbae3..TDbAeNumericMaskProperty
 0001:00002698       ovcdbae3..TOvcfrmDbAeNumericMask
 0001:00002E28       ovcdbae3.Finalization
 0002:0000025C       ovcdbae3.ovcdbae3
 0001:00002A04       ovcdbae3.TDbAeNumericMaskProperty.AllEqual
 0001:00002A08       ovcdbae3.TDbAeNumericMaskProperty.Edit
 0001:000029F8       ovcdbae3.TDbAeNumericMaskProperty.GetAttributes
 0001:00002C0C       ovcdbae3.TOvcfrmDbAeNumericMask.FormCreate
 0001:00002E1C       ovcdbae3.TOvcfrmDbAeNumericMask.FormDestroy
 0001:00002D64       ovcdbae3.TOvcfrmDbAeNumericMask.lbMaskClick
 0004:00000024       ovcdbhbd..2
 0001:00002EC0       ovcdbhbd..TOvcDbBDEHelper
 0001:000032B8       ovcdbhbd.Finalization
 0002:0000026C       ovcdbhbd.ovcdbhbd
 0001:00002FAC       ovcdbhbd.TOvcDbBDEHelper.FindNearestKey
 0001:00002FD4       ovcdbhbd.TOvcDbBDEHelper.GetAliasDriverName
 0001:00003074       ovcdbhbd.TOvcDbBDEHelper.GetAliasNames
 0001:00003084       ovcdbhbd.TOvcDbBDEHelper.GetAliasPath
 0001:0000313C       ovcdbhbd.TOvcDbBDEHelper.GetIndexDefs
 0001:00003154       ovcdbhbd.TOvcDbBDEHelper.GetIndexField
 0001:00003174       ovcdbhbd.TOvcDbBDEHelper.GetIndexFieldCount
 0001:0000318C       ovcdbhbd.TOvcDbBDEHelper.GetIndexFieldNames
 0001:000031E8       ovcdbhbd.TOvcDbBDEHelper.GetIndexName
 0001:00003244       ovcdbhbd.TOvcDbBDEHelper.GetTableNames
 0001:00003258       ovcdbhbd.TOvcDbBDEHelper.IsChildDataSet
 0001:00003278       ovcdbhbd.TOvcDbBDEHelper.SetIndexFieldNames
 0001:00003298       ovcdbhbd.TOvcDbBDEHelper.SetIndexName
 0004:0000002C       ovcdbtb0..3
 0001:00003A80       ovcdbtb0..TOvcDbTableColumnProperty
 0001:00003664       ovcdbtb0..TOvcfrmDbColEditor
 0001:00004AD0       ovcdbtb0.Finalization
 0002:0000027C       ovcdbtb0.ovcdbtb0
 0001:00003B64       ovcdbtb0.TOvcDbTableColumnProperty.Edit
 0001:00003BE0       ovcdbtb0.TOvcDbTableColumnProperty.GetAttributes
 0001:00003BEC       ovcdbtb0.TOvcfrmDbColEditor.AddCellComponentName
 0001:00003BFC       ovcdbtb0.TOvcfrmDbColEditor.btnApplyClick
 0001:00004050       ovcdbtb0.TOvcfrmDbColEditor.btnCloseClick
 0001:0000406C       ovcdbtb0.TOvcfrmDbColEditor.btnFirstClick
 0001:00004084       ovcdbtb0.TOvcfrmDbColEditor.btnLastClick
 0001:000040A8       ovcdbtb0.TOvcfrmDbColEditor.btnNextClick
 0001:000040D8       ovcdbtb0.TOvcfrmDbColEditor.btnPrevClick
 0001:000040FC       ovcdbtb0.TOvcfrmDbColEditor.btnPropertiesClick
 0001:000044B0       ovcdbtb0.TOvcfrmDbColEditor.ctlColNumberChange
 0001:000044F4       ovcdbtb0.TOvcfrmDbColEditor.ctlColNumberExit
 0001:00004644       ovcdbtb0.TOvcfrmDbColEditor.FormClose
 0001:00004670       ovcdbtb0.TOvcfrmDbColEditor.FormShow
 0001:00004518       ovcdbtb0.TOvcfrmDbColEditor.GetCells
 0001:000046DC       ovcdbtb0.TOvcfrmDbColEditor.RefreshColData
 0001:00004A80       ovcdbtb0.TOvcfrmDbColEditor.SetColNum
 0001:00004AA8       ovcdbtb0.TOvcfrmDbColEditor.SetCols
 0004:00000028       ovcdbtb1..2
 0001:00003328       ovcdbtb1..TOvcfrmProperties
 0001:00003634       ovcdbtb1.Finalization
 0002:00000274       ovcdbtb1.ovcdbtb1
 0001:00003574       ovcdbtb1.TOvcfrmProperties.rgDateOrTimeClick
 0004:00000030       ovcregbd..1
 0001:00004B30       ovcregbd.Finalization
 0002:00000284       ovcregbd.ovcregbd
 0001:00004B00       ovcregbd.Register
 0004:00000034       ovcregdb..1
 0001:00004B60       ovcregdb..TOvcDbTableEditor
 0001:00005124       ovcregdb.Finalization
 0002:0000028C       ovcregdb.ovcregdb
 0001:00004CD8       ovcregdb.Register
 0001:00004BE0       ovcregdb.TOvcDbTableEditor.ExecuteVerb
 0001:00004CA0       ovcregdb.TOvcDbTableEditor.GetVerb
 0001:00004CD0       ovcregdb.TOvcDbTableEditor.GetVerbCount
 0001:00000B4C       SysInit.@InitPkg
 0001:00000BB0       SysInit.@PackageLoad
 0001:00000BBC       SysInit.@PackageUnload
 0001:00000A3C       SysInit.AllocTlsBuffer
 0001:00000AF8       SysInit.ExitProcessTLS
 0001:00000AC0       SysInit.ExitThreadTLS
 0001:00000A04       SysInit.FreeLibrary
 0001:00000A48       SysInit.GetTlsSize
 0004:0000000C       SysInit.HInstance
 0001:00000B1C       SysInit.InitializeModule
 0001:00000A94       SysInit.InitProcessTLS
 0001:00000A50       SysInit.InitThreadTLS
 0001:00000A0C       SysInit.LocalAlloc
 0001:00000A14       SysInit.LocalFree
 0003:00000004       SysInit.Module
 0004:00000008       SysInit.ModuleIsLib
 0004:00000009       SysInit.ModuleIsPackage
 0001:00000A1C       SysInit.TlsAlloc
 0004:00000010       SysInit.tlsBuffer
 0001:00000A24       SysInit.TlsFree
 0001:00000A2C       SysInit.TlsGetValue
 0003:00000000       SysInit.TlsIndex
 0005:00000000       SysInit.TlsLast
 0003:0000001C       SysInit.TlsProc
 0001:00000A34       SysInit.TlsSetValue
 0001:00000B28       SysInit.UninitializeModule
 0004:00000000       Windows..3
 0001:00000150       Windows.AnsiToOem
 0001:00000160       Windows.Finalization
 0001:00000148       Windows.FreeLibrary
 0004:00000004       Windows.HtmlHelpModule
 0001:00000158       Windows.OemToAnsi
 0002:00000008       Windows.Windows


  Address             Publics by Value

 0001:00000148       Windows.FreeLibrary
 0001:00000150       Windows.AnsiToOem
 0001:00000158       Windows.OemToAnsi
 0001:00000160       Windows.Finalization
 0001:00000A04       SysInit.FreeLibrary
 0001:00000A0C       SysInit.LocalAlloc
 0001:00000A14       SysInit.LocalFree
 0001:00000A1C       SysInit.TlsAlloc
 0001:00000A24       SysInit.TlsFree
 0001:00000A2C       SysInit.TlsGetValue
 0001:00000A34       SysInit.TlsSetValue
 0001:00000A3C       SysInit.AllocTlsBuffer
 0001:00000A48       SysInit.GetTlsSize
 0001:00000A50       SysInit.InitThreadTLS
 0001:00000A94       SysInit.InitProcessTLS
 0001:00000AC0       SysInit.ExitThreadTLS
 0001:00000AF8       SysInit.ExitProcessTLS
 0001:00000B1C       SysInit.InitializeModule
 0001:00000B28       SysInit.UninitializeModule
 0001:00000B4C       SysInit.@InitPkg
 0001:00000BB0       SysInit.@PackageLoad
 0001:00000BBC       SysInit.@PackageUnload
 0001:00000C90       ovcdbae0..TOvcfrmDbAeRange
 0001:00000EB8       ovcdbae0..TLocalAE
 0001:00001020       ovcdbae0..TLocalEF
 0001:000011BC       ovcdbae0..TDbAeRangeProperty
 0001:00001294       ovcdbae0.TDbAeRangeProperty.GetAttributes
 0001:000012D8       ovcdbae0.TDbAeRangeProperty.GetValue
 0001:00001330       ovcdbae0.ChangeFromRange
 0001:00001398       ovcdbae0.ChangeToRange
 0001:000013FC       ovcdbae0.GetDecimalPlaces
 0001:0000146C       ovcdbae0.TDbAeRangeProperty.Edit
 0001:00001810       ovcdbae0.Finalization
 0001:00001840       ovcdbae1..TOvcfrmDbAeSimpleMask
 0001:00001A64       ovcdbae1..TDbAeSimpleMaskProperty
 0001:00001B44       ovcdbae1.TOvcfrmDbAeSimpleMask.FormCreate
 0001:00001BA8       ovcdbae1.TOvcfrmDbAeSimpleMask.cbxMaskCharacterChange
 0001:00001C1C       ovcdbae1.TDbAeSimpleMaskProperty.GetAttributes
 0001:00001C28       ovcdbae1.TDbAeSimpleMaskProperty.AllEqual
 0001:00001C2C       ovcdbae1.TDbAeSimpleMaskProperty.Edit
 0001:00001DE4       ovcdbae1.TDbAeSimpleMaskProperty.GetEditLimit
 0001:00001DEC       ovcdbae1.Finalization
 0001:00001E1C       ovcdbae2..TOvcfrmDbAePictureMask
 0001:00002098       ovcdbae2..TDbAePictureMaskProperty
 0001:0000217C       ovcdbae2.TDbAePictureMaskProperty.GetAttributes
 0001:00002188       ovcdbae2.TDbAePictureMaskProperty.AllEqual
 0001:0000218C       ovcdbae2.TDbAePictureMaskProperty.Edit
 0001:00002390       ovcdbae2.TOvcfrmDbAePictureMask.FormCreate
 0001:000025A4       ovcdbae2.TOvcfrmDbAePictureMask.lbMaskClick
 0001:0000265C       ovcdbae2.TOvcfrmDbAePictureMask.FormDestroy
 0001:00002668       ovcdbae2.Finalization
 0001:00002698       ovcdbae3..TOvcfrmDbAeNumericMask
 0001:00002914       ovcdbae3..TDbAeNumericMaskProperty
 0001:000029F8       ovcdbae3.TDbAeNumericMaskProperty.GetAttributes
 0001:00002A04       ovcdbae3.TDbAeNumericMaskProperty.AllEqual
 0001:00002A08       ovcdbae3.TDbAeNumericMaskProperty.Edit
 0001:00002C0C       ovcdbae3.TOvcfrmDbAeNumericMask.FormCreate
 0001:00002D64       ovcdbae3.TOvcfrmDbAeNumericMask.lbMaskClick
 0001:00002E1C       ovcdbae3.TOvcfrmDbAeNumericMask.FormDestroy
 0001:00002E28       ovcdbae3.Finalization
 0001:00002EC0       ovcdbhbd..TOvcDbBDEHelper
 0001:00002FAC       ovcdbhbd.TOvcDbBDEHelper.FindNearestKey
 0001:00002FD4       ovcdbhbd.TOvcDbBDEHelper.GetAliasDriverName
 0001:00003074       ovcdbhbd.TOvcDbBDEHelper.GetAliasNames
 0001:00003084       ovcdbhbd.TOvcDbBDEHelper.GetAliasPath
 0001:0000313C       ovcdbhbd.TOvcDbBDEHelper.GetIndexDefs
 0001:00003154       ovcdbhbd.TOvcDbBDEHelper.GetIndexField
 0001:00003174       ovcdbhbd.TOvcDbBDEHelper.GetIndexFieldCount
 0001:0000318C       ovcdbhbd.TOvcDbBDEHelper.GetIndexFieldNames
 0001:000031E8       ovcdbhbd.TOvcDbBDEHelper.GetIndexName
 0001:00003244       ovcdbhbd.TOvcDbBDEHelper.GetTableNames
 0001:00003258       ovcdbhbd.TOvcDbBDEHelper.IsChildDataSet
 0001:00003278       ovcdbhbd.TOvcDbBDEHelper.SetIndexFieldNames
 0001:00003298       ovcdbhbd.TOvcDbBDEHelper.SetIndexName
 0001:000032B8       ovcdbhbd.Finalization
 0001:00003328       ovcdbtb1..TOvcfrmProperties
 0001:00003574       ovcdbtb1.TOvcfrmProperties.rgDateOrTimeClick
 0001:00003634       ovcdbtb1.Finalization
 0001:00003664       ovcdbtb0..TOvcfrmDbColEditor
 0001:00003A80       ovcdbtb0..TOvcDbTableColumnProperty
 0001:00003B64       ovcdbtb0.TOvcDbTableColumnProperty.Edit
 0001:00003BE0       ovcdbtb0.TOvcDbTableColumnProperty.GetAttributes
 0001:00003BEC       ovcdbtb0.TOvcfrmDbColEditor.AddCellComponentName
 0001:00003BFC       ovcdbtb0.TOvcfrmDbColEditor.btnApplyClick
 0001:00004050       ovcdbtb0.TOvcfrmDbColEditor.btnCloseClick
 0001:0000406C       ovcdbtb0.TOvcfrmDbColEditor.btnFirstClick
 0001:00004084       ovcdbtb0.TOvcfrmDbColEditor.btnLastClick
 0001:000040A8       ovcdbtb0.TOvcfrmDbColEditor.btnNextClick
 0001:000040D8       ovcdbtb0.TOvcfrmDbColEditor.btnPrevClick
 0001:000040FC       ovcdbtb0.TOvcfrmDbColEditor.btnPropertiesClick
 0001:000044B0       ovcdbtb0.TOvcfrmDbColEditor.ctlColNumberChange
 0001:000044F4       ovcdbtb0.TOvcfrmDbColEditor.ctlColNumberExit
 0001:00004518       ovcdbtb0.TOvcfrmDbColEditor.GetCells
 0001:00004644       ovcdbtb0.TOvcfrmDbColEditor.FormClose
 0001:00004670       ovcdbtb0.TOvcfrmDbColEditor.FormShow
 0001:000046DC       ovcdbtb0.TOvcfrmDbColEditor.RefreshColData
 0001:00004A80       ovcdbtb0.TOvcfrmDbColEditor.SetColNum
 0001:00004AA8       ovcdbtb0.TOvcfrmDbColEditor.SetCols
 0001:00004AD0       ovcdbtb0.Finalization
 0001:00004B00       ovcregbd.Register
 0001:00004B30       ovcregbd.Finalization
 0001:00004B60       ovcregdb..TOvcDbTableEditor
 0001:00004BE0       ovcregdb.TOvcDbTableEditor.ExecuteVerb
 0001:00004CA0       ovcregdb.TOvcDbTableEditor.GetVerb
 0001:00004CD0       ovcregdb.TOvcDbTableEditor.GetVerbCount
 0001:00004CD8       ovcregdb.Register
 0001:00005124       ovcregdb.Finalization
 0001:00005974       .O406BD2005.@GetPackageInfoTable
 0001:0000597C       .O406BD2005.@PackageLoad
 0001:00005988       .O406BD2005.@PackageUnload
 0002:00000008       Windows.Windows
 0002:00000244       ovcdbae0.ovcdbae0
 0002:0000024C       ovcdbae1.ovcdbae1
 0002:00000254       ovcdbae2.ovcdbae2
 0002:0000025C       ovcdbae3.ovcdbae3
 0002:0000026C       ovcdbhbd.ovcdbhbd
 0002:00000274       ovcdbtb1.ovcdbtb1
 0002:0000027C       ovcdbtb0.ovcdbtb0
 0002:00000284       ovcregbd.ovcregbd
 0002:0000028C       ovcregdb.ovcregdb
 0002:00000294       .O406BD2005..O406BD2005
 0003:00000000       SysInit.TlsIndex
 0003:00000004       SysInit.Module
 0003:0000001C       SysInit.TlsProc
 0004:00000000       Windows..3
 0004:00000004       Windows.HtmlHelpModule
 0004:00000008       SysInit.ModuleIsLib
 0004:00000009       SysInit.ModuleIsPackage
 0004:0000000C       SysInit.HInstance
 0004:00000010       SysInit.tlsBuffer
 0004:00000014       ovcdbae0..5
 0004:00000018       ovcdbae1..3
 0004:0000001C       ovcdbae2..3
 0004:00000020       ovcdbae3..3
 0004:00000024       ovcdbhbd..2
 0004:00000028       ovcdbtb1..2
 0004:0000002C       ovcdbtb0..3
 0004:00000030       ovcregbd..1
 0004:00000034       ovcregdb..1
 0005:00000000       SysInit.TlsLast


Bound resource files

ovcdbae0.DFM
ovcdbae1.DFM
ovcdbae2.DFM
ovcdbae3.DFM
ovcdbtb1.DFM
ovcdbtb0.DFM
OVCREGBD.RES
OVCREGDB.RES
O406BD2005.res
O406BD2005.drf


Program entry point at 0002:00000294
